:020000040800F2
:10000000280B0020E912000811050008130500085C
:10001000170500081B0500081F0500080000000068
:1000200000000000000000000000000023050008A0
:100030002505000800000000270500082905000824
:100040000313000803130008031300080313000838
:100050000313000803130008031300080313000828
:100060000313000803130008031300080313000818
:100070000313000803130008031300080313000808
:1000800003130008031300080313000803130008F8
:1000900003130008031300080313000803130008E8
:1000A00003130008031300080313000803130008D8
:1000B00003130008031300080313000803130008C8
:1000C00003130008031300080313000803130008B8
:1000D000031300081B120008031300080313000891
:1000E0000313000803130008031300080313000898
:1000F0000313000803130008031300080313000888
:100100000313000803130008031300080313000877
:100110000313000803130008031300080313000867
:100120000313000803130008031300080313000857
:1001300000F002F800F063F80AA090E8000C824496
:100140008344AAF10107DA4501D100F058F8AFF273
:10015000090EBAE80F0013F0010F18BFFB1A43F0A5
:1001600001031847B83F0000D83F000010F8013BDA
:100170000A4413F0030408BF10F8014B1D1108BF17
:1001800010F8015B641E05D010F8016B641E01F8C5
:10019000016BF9D1002D15D010F8014B03F00C03C1
:1001A0000C2BA1EB04040ABF10F8013BA4EB831451
:1001B000A4EB032405F1010314F8016B5B1E01F8A5
:1001C000016BF9D5914238BF10F8013BD1D370478C
:1001D0000023002400250026103A28BF78C1FBD850
:1001E000520728BF30C148BF0B607047642902F036
:1001F000FF87002070471FB51FBD10B510BD03F06D
:100200008FF91146FFF7F7FF00F0BDF803F0ADF9E5
:1002100003B4FFF7F2FF03BC00F088FF08B501212B
:10022000082001F00BFC8020ADF8000028208DF89C
:10023000030003208DF8020069469F4801F042F94F
:1002400008BD00B585B00121084601F004FC01217C
:100250000C2001F0F3FB4FF48060ADF8100010208B
:100260008DF8130003208DF8120004A9924801F0C4
:1002700029F94FF40060ADF8100004208DF8130048
:1002800004A98D4801F01EF94FF0804002F066F895
:100290004FF6FF70ADF8040040F26710ADF80000B3
:1002A0000020ADF80600ADF8020069464FF080402E
:1002B00002F028F90121880702F046FF1C208DF882
:1002C0000C0000208DF80D0003208DF80E00012099
:1002D0008DF80F0003A801F02CF805B000BD70B533
:1002E0000025012075490860142000F0CEFE002092
:1002F0007349C1F8A80100214FF0804002F0F2FEDE
:1003000000BF09E0681C05464EF66021884200D90E
:1003100007E0012000F0B9FE68487C38006800283A
:10032000F0D000BF0121880702F048FC002508E05A
:10033000681C05466349884200D907E0012000F0A7
:10034000A4FE5E487C3800680028F1D100BF00217F
:100350004FF0804002F032FC4FF0804002F0E5FEAA
:1003600000EB800000EB001040004FF4FA6190FBBE
:10037000F1F400214FF0804002F0B4FEC82C00D907
:10038000C824A0B270BD4FF4A06000F0CDFF00F013
:1003900063FE00F01BFD4FF4165000F0D6FE00F097
:1003A000FDF900F085FC00F01AFBFFF737FF00F0C5
:1003B000EEFDFFF746FF7EE04348006880B9052068
:1003C00000F087FE4048006850B94048007880F04F
:1003D00001003E49087000BF3B4800680028FBD080
:1003E0003B480078401CC0B23949087064281EDDC3
:1003F0000020087000F0E3FD364908800846B0F997
:1004000000000A2190FBF1F201FB12043148B0F91F
:10041000000090FBF1F523462A462FA1324802F056
:10042000ABFE1023304A0221002000F0B2FB23482B
:100430008C380068E0B92D480078401CC0B22B49C8
:10044000087014281DDDFFF74AFF29490880084677
:100450000088042804DD002018490C31086003E0FE
:10046000012016490C31086001202249087008E07B
:1004700000201E4908701F49087001200F490C31E7
:1004800008601248007848B100200C490831086023
:10049000102319A2042100F07CFB09E00120074988
:1004A00008310860102317A20421002000F071FB1E
:1004B000052000F00EFE7FE7000C0140A8812142DC
:1004C00000802142C02709000001214202000020D3
:1004D000030000200A00002074656D703A25326424
:1004E0002E25316400000000840400200400002058
:1004F00006000020050000206865617465723A6F8F
:100500006E2000006865617465723A6F666600006F
:10051000704700BFFEE700BFFEE700BFFEE700BF79
:10052000FEE7704770477047704700000CB5002029
:10053000019000906C48006840F480306A4908607F
:1005400000BF6948006800F4003000900198401C2A
:100550000190009818B90198B0F5A06FF1D16248E8
:10056000006800F4003010B10120009001E000208C
:1005700000900098012843D15C48006840F01000CA
:100580005A4908600846006820F0030008600846E1
:10059000006840F0020008605348406852494860D3
:1005A0000846406848600846406840F480604860FB
:1005B0000846406820F47C1048600846406840F4D3
:1005C000E81048600846006840F08070086000BF8E
:1005D0004548006800F000700028F9D042484068A3
:1005E00020F00300404948600846406840F002009F
:1005F000486000BF3C48406800F00C000828F9D172
:100600000CBD10B5FFF792FF10BD10B5364800685D
:1006100040F0010034490860084640683449084009
:100620003149486008460068324908402E49086050
:100630000846006820F4802008600846406820F4DE
:10064000FE0048604FF41F008860FFF7DAFF4FF0AC
:1006500000602949086010BD10B50021002000226B
:10066000214B5B6803F00C0121B1042906D0082955
:1006700028D107E0214B224C236027E01F4B204C60
:10068000236023E0184B5B6803F47010164B5B6823
:1006900003F48032022303EB904022B9194B434309
:1006A000174C23600DE0104B5B6803F4003323B15B
:1006B000144B4343124C236003E0104B4343104C54
:1006C000236003E00D4B0E4C236000BF00BF064BC0
:1006D0005B68C3F303130C4CE15C094B1B68CB4014
:1006E000074C236010BD00000010024000200240B3
:1006F0000000FFF8FFFFF6FE08ED00E000127A00B0
:100700001000002000093D001400002008B5012160
:100710004FF4017001F092F94FF4004001F0F2F84B
:100720000F20ADF8000000208DF8030069462A482C
:1007300000F0C8FE08BD00B585B0284801F0E6FB12
:10074000002000908DF804008DF805004FF4602023
:1007500002900020039001208DF8100069461F4888
:1007600001F0FBFB01211D4801F023FC1B4801F0B7
:1007700042FC00BF194801F043FC0028FAD1174899
:1007800001F048FC00BF154801F049FC0028FAD1EF
:100790000121124801F04DFC05B000BD10B5FFF776
:1007A000B5FFFFF7C8FF10BD10B5044607230122AF
:1007B00021460A4801F069FC0121084801F039FC92
:1007C00000BF0221054801F0A5FD0028F9D003482B
:1007D00001F0C2FC10BD00000008014000240140EF
:1007E00010B54FF48051F94800F019FF4FF4005153
:1007F000F64800F014FF4FF40051F44800F011FFE8
:100800004FF48051F14800F00CFF10BD10B54FF4CB
:100810008051EE4800F003FF4FF40051EB4800F028
:1008200000FF4FF40051E94800F0F9FE10BD10B58B
:100830004FF48051E54800F0F2FE4FF48051E34858
:1008400000F0EFFE10BD2DE9F04105462C464FF4B7
:100850008051DE4800F0E5FE00261CE0274607F048
:100860008007802F04D1B901D84800F0D8FE04E0F9
:100870004FF40051D54800F0D4FE6006040E4FF44A
:100880008051D24800F0CBFE4FF48051CF4800F0A9
:10089000C8FE701CC6B2082EE0DBBDE8F08110B5C2
:1008A0000446FFF79DFF7820FFF7CDFFFFF7BFFF5E
:1008B0000020FFF7C8FFFFF7BAFF2046FFF7C3FF8E
:1008C000FFF7B5FFFFF7A2FF10BD10B50446FFF715
:1008D00087FF7820FFF7B7FFFFF7A9FF4020FFF75A
:1008E000B2FFFFF7A4FF2046FFF7ADFFFFF79FFF22
:1008F000FFF78CFF10BD70B504460D461DB1E0B288
:10090000FFF7E3FF02E0E0B2FFF7C9FF70BD70B58B
:100910000646002418E004F1B0000021FFF7EBFFC9
:1009200000210846FFF7E7FF00211020FFF7E3FF53
:10093000002505E001213046FFF7DDFF681CC5B248
:10094000802DF7DB601CC4B2082CE4DB70BD06E030
:1009500041F6650100E0491E0029FCD1401E002837
:10096000F6D17047014605E0002001E0421CD0B2FC
:100970007B28FBDB0A1EA1F10101F5D1704770B5A0
:1009800004460D4605F1B0000021FFF7B4FF102129
:1009900041EA14100021FFF7AEFF04F00F00002120
:1009A000FFF7A9FF70BD10B500218D20FFF7A3FF51
:1009B00000211420FFF79FFF0021AF20FFF79BFFCE
:1009C00010BD10B500218D20FFF795FF00211020EC
:1009D000FFF791FF0021AE20FFF78DFF10BD70B52E
:1009E000002418E004F1B0000021FFF784FF00218B
:1009F0000846FFF780FF00211020FFF77CFF00254D
:100A000005E001210020FFF776FF681CC5B2802DAC
:100A1000F7DB601CC4B2082CE4DB70BD70B50024A9
:100A200018E004F1B0000021FFF765FF002108463F
:100A3000FFF761FF00211020FFF75DFF002505E0B3
:100A400001210846FFF757FF681CC5B2802DF7DB70
:100A5000601CC4B2082CE4DB70BD2DE9F0470746EA
:100A60000E469046994600250024A8F12000C5B204
:100A70007F2F02DD0027B01CC6B2B9F1100F24D1C0
:100A800031463846FFF77BFF002408E004EB0511F0
:100A90004F4A505C0121FFF72EFF601CC4B2082CA6
:100AA000F4DB701CC1B23846FFF769FF002409E08F
:100AB00004EB05110831464A505C0121FFF71BFF8A
:100AC000601CC4B2082CF3DB12E031463846FFF755
:100AD00056FF00240AE005EB45013E4A02EB4101C6
:100AE000085D0121FFF707FF601CC4B2062CF2DB92
:100AF000BDE8F08710B50246012000E050430B1E10
:100B0000A1F10104E1B2F9D110BD2DE9FF5F074663
:100B100091461E460E9D4FF0000A002435E0301B22
:100B2000401EC1B20A20FFF7E5FFB9FBF0F00A2131
:100B3000B0FBF1F201FB1208BAF1000F14D1701EE4
:100B4000A04211DDB8F1000F0CD1AB4605EBDB7113
:100B5000491001FB0471C8B22B4620220199FFF70E
:100B60007CFF10E04FF0010AAB4605EBDB7149104A
:100B700001FB0471C8B208F13001CAB22B460199D9
:100B8000FFF76BFF00BF601CC4B2B442C7DBBDE817
:100B9000FF9F2DE9F04104460F4615469846002672
:100BA0000FE0AA5D434639462046FFF756FF04F1A1
:100BB0000800C4B2782C02DD0024B81CC7B2701C37
:100BC000C6B2A85D0028ECD1BDE8F081000C014060
:100BD0002C3B0008043900082DE9F04180460E4600
:100BE0001546002731464046FFF7C9FE00240AE0BB
:100BF000744A02EB8511085D0121FFF77CFE781C29
:100C0000C7B2601CC4B2102CF2DB701CC1B24046EB
:100C1000FFF7B5FE00240CE06900491C694A02EBAD
:100C20004111085D0121FFF766FE781CC7B2601C08
:100C3000C4B2102CF0DBBDE8F0812DE9F05F064670
:100C40000F4690461C46DDF828A04FF0000BE11738
:100C500004EB5171C910A4EBC10131B92046E11771
:100C600004EB5171C1F3C70506E02046E11704EB20
:100C70005171C910491CCDB23D4615E02946304698
:100C8000FFF77DFEB1460BE059460BF1010B1AF858
:100C900001000121FFF72FFE09F1010000F0FF091B
:100CA000C145F1DB681CC5B2A542E7DBBDE8F09F9A
:100CB00008B50121082000F0C1FE4FF44050ADF806
:100CC000000010208DF8030003208DF80200694613
:100CD0003D4800F0F7FB4FF440513B4800F09FFCCB
:100CE0004FF4487000F0F5F90021AE20FFF703FE45
:100CF00000210846FFF7FFFD00211020FFF7FBFD54
:100D000000214020FFF7F7FD0021B020FFF7F3FDA1
:100D100000218120FFF7EFFD0021FF20FFF7EBFD11
:100D20000021A120FFF7E7FD0021A620FFF7E3FD4A
:100D30000021A820FFF7DFFD00213F20FFF7DBFDAA
:100D40000021C820FFF7D7FD0021D320FFF7D3FDF6
:100D500000210846FFF7CFFD0021D520FFF7CBFD8E
:100D600000218020FFF7C7FD0021D820FFF7C3FD39
:100D700000210520FFF7BFFD0021D920FFF7BBFDB3
:100D80000021F120FFF7B7FD0021DA20FFF7B3FDC6
:100D900000211220FFF7AFFD0021DB20FFF7ABFDA4
:100DA00000213020FFF7A7FD00218D20FFF7A3FDD4
:100DB00000211420FFF79FFD0021AF20FFF79BFDCE
:100DC00008BD000024000020000C014008B50121EE
:100DD000182000F033FE4FF4C040ADF800001020A2
:100DE0008DF8030003208DF802006946084800F0E2
:100DF00069FB4FF48040ADF8000010208DF803002F
:100E000003208DF802006946024800F05BFB08BD34
:100E100000100140000C014008B54FF40070ADF81F
:100E2000000010208DF8030003208DF802006946B1
:100E3000854800F047FB08BD10B5FFF7EDFF002027
:100E40008249086040F2EE2000F01FF9012080493D
:100E5000C1F8A4010F2000F018F910BD08B54FF437
:100E60000070ADF8000028208DF803006946764830
:100E700000F028FB08BD10B50024FFF7EFFF04E0E9
:100E8000601CC4B2012000F000F97048803800688E
:100E900008B1C82CF4DBC82C01DB012010BD0024F4
:100EA00004E0601CC4B2012000F0EFF8674880380D
:100EB000006808B9F02CF4DBF02C01DB0120EDE731
:100EC0000020EBE710B5FFF7A7FF00205F4908609F
:100ED000022000F0DAF801205D49C1F8A401FFF713
:100EE000BDFF0C2000F0D1F858488038006808B1E8
:100EF000012400E00024322000F0C7F8204610BD95
:100F000070B50026012508E0FFF7DCFF0446E0018C
:100F100040EA6600C6B2681CC5B2082DF4DD304652
:100F200070BD70B50446FFF777FF012520E004F09F
:100F3000010664106EB1002044490860022000F0F0
:100F4000A4F801204249C1F8A4013C2000F09DF81A
:100F50000CE000203D4908603C2000F096F801209C
:100F60003B49C1F8A401022000F08FF8681CC5B20B
:100F7000082DDCDD70BD10B5FFF75EFFFFF77BFFCE
:100F8000CC20FFF7CEFF4420FFF7CBFF10BD08B504
:100F90000121092000F052FD4FF40070ADF800006F
:100FA00010208DF8030003208DF8020069462648C2
:100FB00000F088FAFFF740FFFFF75DFF08BD2DE95D
:100FC000F84FFFF7D8FFFFF737FFFFF754FFCC20AC
:100FD000FFF7A7FFBE20FFF7A4FFFFF791FF8346AF
:100FE000FFF78EFF0446072C08DDE043C4B26FEA2A
:100FF0000B0000F0FF0B4FF0000A01E04FF0010A78
:10100000A1464FEA09200FFA80F909EB0B000FFA0D
:1010100080F9484602F018FC009002F0E9FB074610
:1010200000220C4B02F0E6FA054602F0B3FA0FFA82
:1010300080F9BAF1000F02D04846BDE8F88FC9F137
:10104000000000B2F9E70000000C0140A481214239
:10105000008021420000E43F10B56FF0040000F072
:10106000B2F92E4800682E49B0FBF1F02D49087006
:101070000846007800EB4001C1EBC0104FF6FF714D
:1010800001EAC0002849088010BD0146254A1278AF
:101090004A434FF0E0235A6100229A611A461269CE
:1010A00042F001021A6100BF4FF0E022106900F027
:1010B00001021AB100F48032002AF5D04FF0E0228C
:1010C000126922F001024FF0E0231A6100229A61B6
:1010D00070470146144A12884A434FF0E0235A6190
:1010E00000229A611A46126942F001021A6100BF99
:1010F0004FF0E022106900F001021AB100F48032D2
:10110000002AF5D04FF0E022126922F001024FF0E0
:10111000E0231A6100229A6170470000100000204D
:1011200000127A006404002066040020014600BF1B
:10113000704700BF614A128802F04002002AF9D0CD
:10114000C2B25E4B1B1D1A80704710B586B00446B4
:10115000012144F2040000F071FC4FF40070ADF87E
:10116000140003208DF8160018208DF8170005A92B
:10117000534800F0A7F94FF48060ADF81400042044
:101180008DF8170005A94E4800F09CF925208DF830
:10119000000003208DF801008DF8020001208DF879
:1011A0000300684600F0C5F801940020ADF808007F
:1011B000ADF80A00ADF80C00ADF810000C20ADF849
:1011C0000E0001A93D4800F0E0FC012240F224415C
:1011D0003A4800F072FD012240F22551374800F0F4
:1011E0006CFD0121354800F05CFD06B010BD70B506
:1011F00004460D460BE000BF4021304800F02CFEB5
:101200000028F9D014F8011B2C4800F0B7FD281E67
:10121000A5F10101CDB2EED170BD70B540F22551FE
:10122000264800F02FFEA0B1244800F0ABFDC4B268
:1012300024480068312804D22348224909684454CC
:1012400002E000201F4908601E480068401C1D493C
:10125000086040F22441194800F014FE00282CD008
:1012600016480088C5B21548001D0088C5B215484B
:10127000006805281AD915A1134802F07CF818B1A6
:1012800001201449087011E010A10F4802F073F812
:1012900018B100200F49087008E00FA10A4802F0B9
:1012A0006AF818B90EA1084802F065F8002005494F
:1012B00008603121044802F070F870BD0038014028
:1012C0000008014068040020940400206F70656EDF
:1012D00000000000020000206D6F64653100000016
:1012E0006D6F646530000000094880470948004779
:1012F000FEE7FEE7FEE7FEE7FEE7FEE7FEE7FEE7C6
:10130000FEE7FEE704480549054A064B7047000022
:101310000B0600083101000828050020280B0020DA
:10132000280700202807002031490143314A116075
:10133000704770B5002100230F22C47804B32D4CF0
:10134000246804F4E064C4F5E064210AC1F10403F4
:10135000CA40447804FA03F1847814402143090117
:10136000254C0678A155047804F01F050124AC40F3
:1013700005786D11AD0005F1E025C5F8004109E0E3
:10138000047804F01F050124AC401C4D067876114A
:1013900045F8264070BD1A4A0A400243154B1B1FF0
:1013A0001A60704739B1134A121D12680243114B7B
:1013B0001B1D1A6006E00F4A121D126882430D4B76
:1013C0001B1D1A607047042808D14FF0E0210969FD
:1013D00041F004014FF0E022116107E04FF0E021FD
:1013E000096921F004014FF0E0221161704700000B
:1013F0000000FA050CED00E000E400E080E100E010
:1014000080FFFF1F10B50446CC48844208D101215B
:10141000042000F02DFB0021042000F029FB46E011
:10142000C748844208D10121082000F021FB002197
:10143000082000F01DFB3AE0C248844208D1012197
:10144000102000F015FB0021102000F011FB2EE011
:10145000BD48844208D10121202000F009FB002171
:10146000202000F005FB22E0B848844208D1012189
:10147000402000F0FDFA0021402000F0F9FA16E0CB
:10148000B348844208D10121802000F0F1FA002104
:10149000802000F0EDFA0AE0AE48844207D1012135
:1014A000801500F0E5FA0021A01500F0E1FA10BD6A
:1014B00010B50121084600F0DBFA0021012000F000
:1014C000D7FA10BD2DE9F041024600250026002084
:1014D00000230024002791F803C00CF00F0591F8B9
:1014E00003C00CF0100CBCF1000F03D091F802C047
:1014F0004CEA050591F800C0BCF1000F31D014682A
:1015000000202BE04FF0010C0CFA00F3B1F800C002
:101510000CEA03069E4220D183004FF00F0C0CFA18
:1015200003F7BC4305FA03FC4CEA040491F803C03A
:10153000BCF1280F06D14FF0010C0CFA00FCC2F8E8
:1015400014C00AE091F803C0BCF1480F05D14FF078
:10155000010C0CFA00FCC2F810C0401C0828D1D3C2
:101560001460B1F800C0BCF1FF0F34DD54680020F6
:101570002EE000F1080C4FF0010808FA0CF3B1F866
:1015800000C00CEA03069E4221D183004FF00F0CED
:101590000CFA03F7BC4305FA03FC4CEA040491F887
:1015A00003C0BCF1280F05D100F1080C08FA0CF8B3
:1015B000C2F8148091F803C0BCF1480F07D100F1C4
:1015C000080C4FF0010808FA0CF8C2F81080401C13
:1015D0000828CED35460BDE8F0814FF6FF7101803A
:1015E000022181700421C170704702460020936877
:1015F0000B400BB1012000E00020704701468868D5
:1016000080B2704702460020D3680B400BB1012026
:1016100000E0002070470146C86880B27047016151
:101620007047416170470AB1016100E04161704754
:10163000C16070474FF480320A43826181618261E8
:1016400082698269704702460020434B18684FF652
:101650008073184040EA021008433F4B18607047FF
:101660003E49C8617047F0B50A46002300240021B6
:10167000002500F00046B6F1004F02D1364EF16968
:1016800001E0354E7168C0F3034583B200F44016A3
:10169000B6F5401F08D121F070612F4E766826F014
:1016A00070662D4F7E6012E000F48016B6F5801F44
:1016B00006D1032606FA05F4A14341F0706106E065
:1016C000460D360103FA06F6B14341F0706122B1CE
:1016D000460D360103FA06F6314300F00046B6F136
:1016E000004F02D11C4EF16101E01B4E7160F0BD54
:1016F00030B500228B071C0F0F2303FA04F2164BA0
:1017000008338C1053F824309343134C08348D1055
:1017100044F8253023468C1053F824308C07240FCE
:1017200000FA04F423430C4C08348D1044F825309F
:1017300030BD0A49DC3108607047000000080140F4
:10174000000C01400010014000140140001801404D
:10175000001C014000200140000001400000204228
:10176000DF48006840F00100DD4908600846406835
:10177000DC490840DA49486008460068DA49084010
:10178000D74908600846006820F4802008600846B1
:10179000406820F4FE0048604FF41F0088607047E6
:1017A000CF49096821F48031CD4A1160114609689A
:1017B00021F480211160B0F5803F03D0B0F5802F77
:1017C0000ED106E0C649096841F48031C44A11606F
:1017D00007E0C349096841F4A021C14A116000E053
:1017E00000BF00BF704710B5014600220023002053
:1017F0004A11012A02D1BA4C236806E0022A02D11A
:10180000B74C236A01E0B64C636A01F01F02012461
:1018100094401C400CB1012000E0002010BD38B500
:10182000002000900024002500BF3120FFF7DBFFDF
:1018300005460098401C00900098B0F5A06F01D0BC
:10184000002DF2D03120FFF7CEFF08B1012400E0D7
:101850000024204638BD01460020A14A106820F02F
:10186000F80040EAC10010607047A0490860704766
:10187000024600209A4B586820F47C1042EA01038B
:101880001843974B5860704798490866704701465F
:101890000020934A506820F00300084350607047CE
:1018A0008F48406800F00C007047014600208C4AC9
:1018B000506820F0F0000843506070470146002057
:1018C000874A506820F4E060084350607047014642
:1018D0000020834A506820F4605040EAC100506004
:1018E000704729B17E4A527A02437D4B5A7204E016
:1018F0007B4A527A82437A4B5A7270477B49D8317D
:101900000860704701460020754A506820F4404046
:101910000843506070470021714A20321170704AAC
:1019200082F82010012802D004280AD104E0012105
:101930006B4A2032117005E00521694A203211708E
:1019400000E000BF00BF7047694908607047644904
:10195000096A0143624A1162704765494439086067
:10196000704730B500210022002400235C4D6D68D3
:1019700005F00C0121B1042905D0082923D105E087
:101980005C4D056022E05B4D05601FE0544D6D68C5
:1019900005F47012524D6D6805F48034022505EB94
:1019A00092421CB9544D554305600BE04C4D6D6897
:1019B00005F400351DB1504D5543056002E04D4D15
:1019C0005543056002E04B4D056000BF00BF444D2C
:1019D0006D6805F0F0010909484D6B5C0568DD4054
:1019E00045603F4D6D6805F4E061090A434D6B5C4D
:1019F0004568DD4085603A4D6D6805F46051C90A5F
:101A00003E4D6B5C4568DD40C560354D6D6805F445
:101A10004041890B3A4D6B5CC568B5FBF3F5056138
:101A200030BD29B12E4A526902432D4B5A6104E060
:101A30002B4A526982432A4B5A61704729B1284A7E
:101A400092690243264B9A6104E0254A92698243D7
:101A5000234B9A61704729B1214AD2690243204B36
:101A6000DA6104E01E4AD26982431D4BDA61704795
:101A700029B11B4AD2680243194BDA6004E0184AC4
:101A8000D2688243164BDA60704729B1144A126952
:101A90000243134B1A6104E0114A12698243104B4E
:101AA0001A61704712494039086070470F49C8648D
:101AB00070470B49C87170470948406A40F0807010
:101AC00007494862704701460020054A92680A406B
:101AD0000AB1012000E00020704701498872704778
:101AE000001002400000FFF8FFFFF6FE0000424237
:101AF0008004424200127A0000093D007004002078
:101B00008004002010B50446FB48844209D101211D
:101B10008803FFF7ADFF00214FF48040FFF7A8FFD7
:101B200032E0F648844209D101214804FFF7ADFFB5
:101B300000214FF40030FFF7A8FF25E0F048844271
:101B400009D101218804FFF7A0FF00214FF4802074
:101B5000FFF79BFF18E0EB48844209D10121C8043C
:101B6000FFF793FF00214FF40020FFF78EFF0BE0FB
:101B7000E548844208D101210805FFF786FF0021CE
:101B80004FF48010FFF781FF10BD2DE9F04786B0BC
:101B900005460E460024A24600BFA1460027B08994
:101BA00000B100BF2F462C8A4CF6FF700440F0882D
:101BB00004432C82AC894EF6F3100440B08831897E
:101BC0000843718908430443AC81AC8A4FF6FF4057
:101BD0000440B0890443AC8201A8FFF7C2FEC648A6
:101BE000874202D1DDF810A001E0DDF80CA0A88941
:101BF00000F4004040B10AEBCA0000EB0A10316863
:101C00004900B0FBF1F807E00AEBCA0000EB0A104C
:101C100031688900B0FBF1F86420B8FBF0F00401F2
:101C20002009642101FB1089A88900F4004040B11B
:101C3000322000EBC900B0FBF1F000F007000443D4
:101C400008E0322000EB09106421B0FBF1F000F055
:101C50000F0004432C8106B0BDE8F0874FF4165105
:101C6000016000218180C18001810C21418100211E
:101C70008181704710B502460020108A4FF2FF03A1
:101C800018400B884C8823438C882343CC882343FB
:101C90001843108210BD0021018041808180C180E5
:101CA000704721B1828942F40052828104E0828926
:101CB0004DF6FF731A4082817047F0B50346002449
:101CC00000260025002040F66A17B94200D100BF67
:101CD0001846C1F3421401F01F06012707FA06F562
:101CE000012C01D10C3004E0022C01D1103000E0B5
:101CF00014301AB107682F43076002E00768AF434A
:101D00000760F0BD1AB1838A0B43838202E0838AA5
:101D10008B4383827047028A4FF6F0731A40028227
:101D2000028A0A430282704782894FF2FF731A4087
:101D3000828182890A438281704721B1828942F07F
:101D40000202828104E082894FF6FD731A4082818B
:101D50007047028A4FF6DF731A400282028A0A43F2
:101D60000282704721B1028A42F48042028204E07A
:101D7000028A4BF6FF731A4002827047C1F30802D1
:101D80008280704701468888C0F3080070478189C7
:101D900041F0010181817047028BD2B20283028B34
:101DA00042EA012202837047028B02F47F420283DF
:101DB000028B0A430283704721B1828A42F02002DB
:101DC000828204E0828A4FF6DF731A408282704773
:101DD00021B1828A42F01002828204E0828A4FF6A8
:101DE000EF731A408282704721B1828A42F0080262
:101DF000828204E0828A4FF6F7731A40828270472B
:101E000021B1828942F40042828103E08289C2F3D7
:101E10000E028281704721B1828A42F4006282827E
:101E200004E0828A4FF2FF731A4082827047828AEE
:101E30004FF6FB731A408282828A0A43828270477D
:101E400021B1828A42F00202828204E0828A4FF645
:101E5000FD731A408282704702460020B1F5007F70
:101E600000D100BF13880B400BB1012000E000201F
:101E7000704701F40072B2F5007F00D100BFCA4381
:101E80000280704770B50246002400230025002020
:101E900040F66A16B14200D100BFC1F3421501F00D
:101EA0001F03012606FA03F3012D02D19689334060
:101EB00006E0022D02D1168A334001E0968A3340B3
:101EC0000C12012606FA04F41688344013B10CB142
:101ED000012000E0002070BD10B50022002340F674
:101EE0006A14A14200D100BF0A1201249440A3B297
:101EF000DC43048010BD0000003801400044004075
:101F000000480040004C00400050004010B504461E
:101F1000FA48844208D101214015FFF7A9FD0021AC
:101F20006015FFF7A5FD17E0F548844208D10121AF
:101F30000015FFF79DFD00212015FFF799FD0BE02F
:101F4000F048844208D10121C803FFF791FD002128
:101F50004FF40040FFF78CFD10BD30B50246002065
:101F600000235068E84C20400D790C6844EA0524B1
:101F7000204350609068E54C2040D1E902542C4346
:101F80004D7944EA450420439060D06A20F4700003
:101F90000C7C641EE4B2234340EA0350D06230BD9F
:101FA00000210160017141718160C16001210174F2
:101FB000704721B1826842F00102826003E08268CA
:101FC00022F001028260704721B1826842F480727F
:101FD000826003E0826822F480728260704710B5EC
:101FE0000023CBB21AB144681C43446002E0446849
:101FF0009C43446010BD816841F0080181607047D6
:10200000014600208A6802F008020AB1012000E0BF
:1020100000207047816841F00401816070470146EB
:1020200000208A6802F004020AB1012000E00020CA
:10203000704721B1826842F4A002826003E08268A6
:1020400022F4A00282607047014600208A6802F4F0
:1020500080020AB1012000E00020704710B50A4656
:1020600000210023416821F46041531E41EA4331BD
:10207000416010BD21B1426842F40062426003E059
:10208000426822F4006242607047F0B504460D4693
:1020900000200021092D11DDE068A5F10A0606EBFC
:1020A0004607072606FA07F18843A5F10A0606EB5C
:1020B000460603FA06F10843E0600CE0206905EBF0
:1020C0004507072606FA07F1884305EB450603FA9C
:1020D00006F108432061072A0FDA606B561E06EBF3
:1020E00086071F2606FA07F18843561E06EB86066A
:1020F00005FA06F10843606322E00D2A0FDA206B2F
:10210000D61F06EB86071F2606FA07F18843D61F5F
:1021100006EB860605FA06F10843206310E0E06A44
:10212000A2F10D0606EB86071F2606FA07F1884383
:10213000A2F10D0606EB860605FA06F10843E062F9
:10214000F0BD21B1826842F48012826003E08268AF
:1021500022F48012826070470146C86C80B27047DA
:1021600066484C300068704721B1426842F4806292
:10217000426003E0426822F480624260704721B10D
:10218000426842F48052426003E0426822F4805286
:10219000426070470A460021816821F4E041114302
:1021A0008160704721B1826842F40042826003E09E
:1021B000826822F400428260704721B1826842F452
:1021C0000212826003E0826822F402128260704789
:1021D000014600208A6802F400120AB1012000E0E2
:1021E00000207047F0B50446154600200022002666
:1021F000092911DDE068A1F10A0707EB470C072761
:1022000007FA0CF29043A1F10A0707EB470703FA1C
:1022100007F21043E0600CE0206901EB410C072756
:1022200007FA0CF2904301EB410703FA07F210435F
:102230002061A06BC0F30156EF1C06F1010CA7EB67
:102240000C0707EB870C1F2707FA0CF29043EF1CD3
:1022500006F1010CA7EB0C0707EB870701FA07F261
:102260001043A063F0BD10B50A4600210023816B26
:1022700021F44011531E41EA0351816310BD08B59A
:10228000002300930090009B0B440093009B1A6076
:1022900008BD08B5024600200090009201F1280018
:1022A000009B184400900098006880B208BD0A4660
:1022B00000214168164B194011434160704741624B
:1022C000826270470A460021416821F01F011143D4
:1022D0004160704740B109490831096841F4000183
:1022E000064A0832116007E004490831096821F400
:1022F0000001024A083211607047000000240140CA
:1023000000280140003C0140FFFEF0FFFDF7F1FF17
:10231000FFFD3FFF0246002013680B400BB1012078
:1023200000E000207047CA430260704770B5024663
:102330000020002300240B125568CEB205EA0604E3
:1023400015681D4015B10CB1012000E0002070BDE2
:1023500000220A12D34303607047000010B5044600
:10236000FE48844208D10121C014FFF781FB0021FF
:10237000E014FFF77DFBC4E0B4F1804F08D10121E8
:102380000846FFF782FB00210120FFF77EFBB8E043
:10239000F348844208D101210220FFF776FB002197
:1023A0000220FFF772FBACE0EE48844208D1012125
:1023B0000420FFF76AFB00210420FFF766FBA0E082
:1023C000E948844208D101210820FFF75EFB002183
:1023D0000820FFF75AFB94E0E448844208D1012129
:1023E0001020FFF752FB00211020FFF74EFB88E082
:1023F000DF48844208D101212020FFF746FB00215D
:102400002020FFF742FB7CE0DA48844208D101211A
:102410004014FFF72DFB00216014FFF729FB70E04B
:10242000D548844209D10121C804FFF721FB0021CE
:102430004FF40020FFF71CFB63E0D048844209D131
:1024400001210805FFF714FB00214FF48010FFF76E
:102450000FFB56E0CA48844209D101214805FFF725
:1024600007FB00214FF40010FFF702FB49E0C548CD
:10247000844208D101214020FFF707FB00214020C2
:10248000FFF703FB3DE0C048844208D101218020D2
:10249000FFF7FBFA00218020FFF7F7FA31E0BB4895
:1024A000844208D101218015FFF7EFFA0021A01521
:1024B000FFF7EBFA25E0B648844209D10121080470
:1024C000FFF7D6FA00214FF48030FFF7D1FA18E079
:1024D000B048844209D101214804FFF7C9FA00211C
:1024E0004FF40030FFF7C4FA0BE0AB48844208D148
:1024F00001218804FFF7BCFA00214FF48020FFF788
:10250000B7FA10BD00220288944B98420ED0994B26
:1025100098420BD0B0F1804F08D0914B984205D033
:10252000904B984202D0904B984204D14FF68F7353
:102530001A404B881A438D4B984207D08C4B9842D7
:1025400004D04FF6FF431A40CB881A4302808B8891
:1025500083850B880385814B98420BD0854B98422D
:1025600008D08B4B984205D08A4B984202D08A4BB8
:10257000984201D10B7A038601238382704770B59C
:10258000002400220023058C4FF6FE76354005849A
:10259000028C8388048B4FF68F752C40B51E2C401F
:1025A0000D882C43751E2A400D892A434D882A43E5
:1025B0006A4DA8420BD06F4DA84208D0744DA84276
:1025C00005D0744DA84202D0734DA84213D14FF6E6
:1025D000F7752A404D892A434FF6FB752A408D88AE
:1025E0002A434FF6FF652B404FF6FF552B408D8950
:1025F0002B43CD892B4383800483CD888586028439
:1026000070BD70B5002400220023058C4FF6EF76D4
:1026100035400584028C8388048B48F6FF752C4076
:102620004FF6FF452C400D884FF6FF7606EA05254C
:102630002C434FF6DF752A400D8906EA05152A431B
:102640004D8806EA05152A43444DA84202D0494D5B
:10265000A8421DD14FF67F752A404D894FF6FF766F
:1026600006EA05152A434FF6BF752A408D8806EA0B
:1026700005152A434FF6FF352B404FF2FF752B40CF
:102680008D8906EA85052B43CD8906EA85052B430E
:1026900083800483CD880587028470BD70B50024D3
:1026A00000220023058C4FF6FF6635400584028C1E
:1026B0008388848B4FF68F752C404FF6FC752C4029
:1026C0000D882C434FF6FF552A400D894FF6FF76B3
:1026D00006EA05252A434D8806EA05252A431F4DAB
:1026E000A84202D0234DA8421DD14FF2FF752A40C7
:1026F0004D894FF6FF7606EA05252A434FF6FF354A
:102700002A408D8806EA05252A434EF6FF752B40A0
:102710004DF6FF752B408D8906EA05152B43CD89B3
:1027200006EA05152B4383808483CD888587028440
:1027300070BD70B5002200230024058C4EF6FF7694
:1027400035400584038C8488828B48F6FF752A40C7
:102750004FF6FF452A400D8820E00000002C014084
:102760000004004000080040000C00400010004041
:102770000014004000340140004C01400050014072
:102780000054014000180040001C004000200040A0
:102790000040014000440140004801404FF6FF76F0
:1027A00006EA05252A434DF6FF752B400D8906EAFA
:1027B00005352B434D8806EA05352B43FA4DA842D3
:1027C00002D0FA4DA84208D14BF6FF752C408D89F6
:1027D0004FF6FF7606EA85152C4384808283CD88E8
:1027E000A0F84050038470BD828B4FF2FF331A4033
:1027F0008283828B4FF6FF7303EA01231A4382839D
:102800007047F0B50C461546002200210026078CC3
:102810004EF6FF7C07EA0C070784828B018C4FF68B
:10282000FF7707EA043640F6FF473A404FF6FF7756
:1028300007EA05273A434FF6FF7707EA03373A439B
:10284000D94FB8420ED0D94FB8420BD0B0F1804F1B
:1028500008D0D74FB84205D0D64FB84202D0D64F95
:10286000B84206D14DF6FF77394046F480573943D8
:1028700005E047F6FF57394044F4805739438283D7
:102880000184F0BD828B4FF6F3731A408283828BF2
:102890000A4382837047F0B50C461546002200219A
:1028A0000026078C4FF6FF6C07EA0C070784828B23
:1028B000018C4FF6FF7707EA04264FF60C773A4073
:1028C0004FF6FF7707EA03172F433A43B64FB84254
:1028D0000ED0B64FB8420BD0B0F1804F08D0B44FF5
:1028E000B84205D0B34FB84202D0B34FB84206D178
:1028F0004FF6FF57394046F48077394305E04FF2F1
:10290000FF57394044F48077394382830184F0BD16
:10291000028B4FF2FF331A400283028B4FF6FF7394
:1029200003EA01231A4302837047F0B50C461546AB
:10293000002200210026078C4FF6EF7C07EA0C07E7
:102940000784028B018C4FF6FF7707EA041640F6E6
:10295000FF473A404FF6FF7707EA03373A434FF60F
:10296000FF7707EA05273A438F4FB8420ED08F4FC3
:10297000B8420BD0B0F1804F08D08D4FB84205D08F
:102980008C4FB84202D08C4FB84206D14FF6DF7759
:10299000394046F01007394305E04FF65F7739407C
:1029A00044F01007394302830184F0BD028B4FF6D7
:1029B000F3731A400283028B0A4302837047F0B517
:1029C0000C46154600220021068C4FF6FE773E404D
:1029D0000684028B018C4FF60C7632407E1C06EA90
:1029E00003162E433243704EB0420ED06F4EB042AB
:1029F0000BD0B0F1804F08D06D4EB04205D06D4E77
:102A0000B04202D06C4EB04206D14FF6FD76314056
:102A100044F00106314305E04FF6F576314044F0CD
:102A20000106314302830184F0BD70B505460C46B2
:102A30005D4885420ED05D4885420BD0B5F1804F90
:102A400008D05B48854205D05A48854202D05A4892
:102A5000854200D100E000BF208850B92389A288B8
:102A600061882846FFF7ABFFE1882846FFF79EFF05
:102A700025E0208804280AD12389A2886188284675
:102A8000FFF753FFE1882846FFF742FF17E0208851
:102A900008280AD12389A28861882846FFF7FBFE0F
:102AA000E1882846FFF7EEFE09E02389A2886188C5
:102AB0002846FFF7A6FEE1882846FFF795FE70BD81
:102AC0002DE9F04105460C4600260127608808B92B
:102AD000022600E00026A088012801D1022700E09C
:102AE00001272088A0B92389A28861882846FFF79A
:102AF00066FFE1882846FFF759FF23893A463146A9
:102B00002846FFF712FFE1882846FFF701FF13E090
:102B10002389A28861882846FFF707FFE1882846B5
:102B2000FFF7F6FE23893A4631462846FFF747FF6E
:102B3000E1882846FFF73AFFBDE8F0810A884B8814
:102B40001A438B881A43CB881A430B891A434B8943
:102B50001A438B891A43A0F8442070474FF6FF713F
:102B6000818000210180C180418001727047002175
:102B7000018041808180C180018141818181C18149
:102B80007047002101804180012181800021C180A6
:102B9000018170470021018041808180C1800181D5
:102BA0004181818170470000002C014000340140C8
:102BB0000004004000080040000C004021B10288E1
:102BC00042F00102028004E002884FF6FE731A40D0
:102BD0000280704731B1B0F8442042F40042A0F8BE
:102BE000442005E0B0F84420C2F30E02A0F84420CF
:102BF00070471AB183890B43838102E083898B4339
:102C0000838170478182704741EA0203A0F848300F
:102C100070471AB183890B43838102E083898B4318
:102C20008381704701894FF6F87211400181704726
:102C30000A46002101894FF68F7319401143018123
:102C4000704730B504460D4629462046FFF7F0FF91
:102C5000208940F00700208130BD2DE9F041044675
:102C60000D4616461F46602D06D13B4601223146D1
:102C70002046FFF75AFE05E03B460122314620463A
:102C8000FFF79DFE29462046FFF7D2FF208940F03E
:102C900007002081BDE8F08130B50C460021018994
:102CA000C9B24FF6FF7505EA0325154325432943AD
:102CB000018130BD2DE9F04105460E461746984684
:102CC000002443463A4631462846FFF7E5FF2C8963
:102CD0004FF6F870044044F007044FF68F7004403C
:102CE00044F070042C81BDE8F081F0B504460D4637
:102CF00016461F463B46324629462046FFF7CCFF84
:102D0000208940F480402081F0BD01858282704797
:102D10000A46002101884FF68F7319401143018044
:102D20007047F0B50C4615461E46002100220023D0
:102D30000189028B038C4FF6F877394021434FF617
:102D4000FC473A4040F201173A434FF6DD773B40EB
:102D50004FF6FF7707EA06172F433B4301810283B3
:102D60000384F0BD0A460021018B4FF68F73194092
:102D70001143018370470A460021018B48F6FF7317
:102D800019404FF6FF7303EA02231943018370478A
:102D90000A460021818B4FF68F73194011438183BE
:102DA00070470A460021818B48F6FF7319404FF6A1
:102DB000FF7303EA022319438183704721B102881C
:102DC00042F08002028004E002884FF67F731A40CE
:102DD0000280704721B1828842F00402828004E0C0
:102DE00082884FF6FB731A408280704721B1828837
:102DF00042F00802828004E082884FF6F7731A409E
:102E00008280704721B1828842F00102828004E012
:102E100082884FF6FE731A40828070470A4600216E
:102E2000018B4FF6F77319401143018370470A462F
:102E30000021018B4FF2FF7319404FF6FF7303EA35
:102E400002231943018370470A460021818B4FF604
:102E5000F77319401143818370470A460021818B23
:102E60004FF2FF7319404FF6FF7303EA0223194331
:102E7000818370470A460021018B4FF6FB7319408E
:102E80001143018370470A460021018B4FF6FF333F
:102E900019404FF6FF7303EA022319430183704779
:102EA0000A460021818B4FF6FB7319401143818341
:102EB00070470A460021818B4FF6FF3319404FF6C9
:102EC000FF7303EA02231943818370470A460021F6
:102ED000018B4FF67F7319401143018370470A46F7
:102EE0000021018BC1F30E014FF6FF7303EA0223A9
:102EF0001943018370470A460021818B4FF67F7387
:102F000019401143818370470A460021818BC1F328
:102F10000E014FF6FF7303EA0223194381837047C2
:102F20000A460021018C4FF6FD73194011430184BC
:102F300070470A460021018C4FF6F7731940114380
:102F4000018470470A460021018C4FF6DF73194057
:102F50004FF6FF7303EA02131943018470470A46D0
:102F60000021018C4FF67F7319404FF6FF7303EA7F
:102F700002131943018470470A460021018C4FF661
:102F8000FF5319404FF6FF7303EA022319430184EC
:102F900070470A460021018C4FF2FF7319404FF62B
:102FA000FF7303EA02231943018470470A46002194
:102FB000018C4DF6FF7319404FF6FF7303EA02339D
:102FC00019430184704730B5002301248C40A3B21B
:102FD000048C9C430484048C02FA01F5ADB22C43AA
:102FE000048430BD30B5002304248C40A3B2048C8B
:102FF0009C430484048C02FA01F5ADB22C43048492
:1030000030BD70B503460020002418461830012555
:103010008D40ACB21D8CA5431D8409B1082909D18E
:1030200000EB6100056825F0700505600568154333
:1030300005600EE00D1FC5F34E052844056825F414
:10304000E045056005684FF6FF7606EA022635433F
:10305000056070BD21B1028842F00202028004E0E6
:1030600002884FF6FD731A400280704721B1028832
:1030700042F00402028004E002884FF6FB731A401B
:103080000280704721B1828842F08002828004E091
:1030900082884FF67F731A408280704702884FF60D
:1030A000F7731A40028002880A43028070478288C0
:1030B0004FF68F731A40828082880A43828070475D
:1030C00002894FF6F8731A40028102890A4302818D
:1030D000704702894FF67F731A40028102890A43C2
:1030E000028170478184704781857047818670476F
:1030F0000187704781877047A0F8401070470288A9
:103100004FF6FF431A40028002880A43028070474C
:103110000146888E70470146088F70470146888FA8
:1031200070470146B1F8400070470146888C7047EF
:103130000146088D704702460020138A0B400BB1F0
:10314000012000E000207047CA430282704730B57A
:103150000246002000230024158A05EA0103958910
:1031600005EA010413B10CB1012000E0002030BDDC
:10317000CA430282704770470FB41CB5074B06AABA
:103180007B4469460090059800F08BF90020694661
:1031900000F09AF91CBC5DF814FB00004503000028
:1031A00070B5044685690068C10601D5302600E087
:1031B0002026C00707D070BDD4E9012130469047D2
:1031C000206A401C20626D1EF6D570BD70B50446A5
:1031D00085690078C00707D170BDD4E9012120209E
:1031E0009047206A401C20626D1EF6D570BD00001D
:1031F0002DE9F0410646002410687529314616A5D0
:1032000010D0AFF30080002802DA404213A507E097
:1032100031688A0701D512A502E0490704D511A536
:10322000012401E0AFF3008000210A2206F1240707
:1032300009E0B0FBF2FCB0FBF2F302FB1C00303003
:1032400078541846491C0028F3D123462A463046B4
:10325000BDE8F04100F0C7B8000000002D000000FC
:103260002B000000200000002DE9F0474FF0000A7D
:1032700089460446C0F820A02046E1688847002817
:1032800076D0252806D0D4E901219047206A401C39
:103290002062F1E7E168204600258847C4F81CA0B9
:1032A00006460027C4F818A02A2E09D0304600F0A0
:1032B00069F938B304EB8708303EC8F8186019E0A4
:1032C00059F8041B204604EB87029161E1688847A6
:1032D000012F064618D1E069002820DA25F02005E4
:1032E0001DE0D8F8180000EB800006EB40003038F5
:1032F000C8F818002046E1688847064600F042F901
:103300000028EED1012F0AD02E2E08D12046E168E8
:1033100088477F1C0646022F45F02005C4DBA069C4
:10332000002803DA404245F00105A061E80701D01A
:1033300025F01005B6B1A6F14100192802D82036B3
:1033400045F400654A463146204625604D46FCF767
:103350004DFF58B1012806D0ED1D25F0070000F102
:10336000080989E704E005F1040985E730468AE7A2
:10337000206ABDE8F08730B505460B462A4613F8AB
:10338000014B12F8010B08B1A042F8D01CB1002883
:1033900002D06D1CF1E7284630BD4FF00002042931
:1033A000C0F0128010F0030C00F09580CCF1040CFA
:1033B000BCF1020F18BF00F8012BA8BF20F8022BA8
:1033C000A1EB0C0100F087B85FEAC17C24BF00F8D4
:1033D000012B00F8012B48BF00F8012B7047704704
:1033E0007047704770472DE9F0470D469946924661
:1033F000044600F124080168880604D5E06921F03C
:103400001001216000E00120A84201DD471B00E01F
:103410000027A1697A1902EB0900081AA061207837
:10342000C00602D42046FFF7BBFE002608E0D4E920
:1034300001211AF806009047206A401C761C206281
:103440004E45F4DB2078C0060AD52046FFF7A8FEDB
:1034500006E0D4E9012130209047206A401C206218
:10346000381EA7F10107F4DC07E0D4E9012118F8C0
:1034700005009047206A401C2062281EA5F1010526
:10348000F3DC2046FFF7A2FE2078000602D50220DA
:10349000BDE8F0870120FBE701694A1C026108785A
:1034A000704700B58FB0CDE9013100210591054984
:1034B0007944CDE9031011466846FFF7D5FE0FB0F9
:1034C00000BD0000E5FFFFFF0A6802F8010B0A607B
:1034D00070474FF0000200B51346944696462039D7
:1034E00022BFA0E80C50A0E80C50B1F12001BFF4BD
:1034F000F7AF090728BFA0E80C5048BF0CC05DF823
:1035000004EB890028BF40F8042B08BF704748BF70
:1035100020F8022B11F0804F18BF00F8012B7047E4
:10352000754600F02BF8AE4605006946534620F07C
:103530000700854618B020B5FDF7E4FEBDE8204041
:103540004FF000064FF000074FF000084FF0000B5F
:1035500021F00701AC46ACE8C009ACE8C009ACE812
:10356000C009ACE8C0098D46704710B50446AFF3FA
:1035700000802046BDE81040FCF74ABE0048704776
:10358000C804002030380A2801D2012070470020EA
:10359000704700004FEA41034FEA5353A3F580639D
:1035A000D3F11E03C8BFD3F1210C0CDD4FF0004254
:1035B00042EAC12242EA505232FA03FC8CEAE17C30
:1035C000ACEBE1707047102BC4BF0020704703F5CF
:1035D000787CBCF1FF3F04D06FF0004282EA21000A
:1035E000704770B500F0B0F8499224800020704711
:1035F000F2E70000DFF848C170B51CEA111E1EBFDB
:103600001CEA13159EEA0C0F95EA0C0F00F06F8070
:1036100081EA030423EA4C134EEAD47E21EA4C11DA
:1036200041F4801143F48013AE44A1FB024CA0FB93
:103630000365AEF17F7E361955EB0C05A1FB034CFB
:103640004CF10003A0FB021C16EB0C06654153F184
:103650000003094218BF46F0010613F4007F0BD1A6
:103660004FEA03314FEA0530340341EA155140EA8D
:1036700016506FF003020AE04FEAC3214FEAC5205B
:10368000F40241EA555140EA56506FF0020202EB53
:103690002E4201EB025585EACE710AD05FEA440C56
:1036A00018BF24F0004450F1000041F1000120EA6D
:1036B000D47040F2FE7C624500D270BDA84214BFB7
:1036C0004FF080444FF04044002E08BF0024BEF16C
:1036D000806FA8BFA1F1C041BDE8704080F2828038
:1036E0004FF0000001F1C04101F0004170479EEA37
:1036F0000C0F0CEA131518BF95EA0C0F06D04FF00B
:10370000000081EA030E0EF0004170BD00F01CF8CD
:103710008900013E00F007B800F009B84FEA430CF9
:103720005FEA5C5C08D081EA030100F05BB84FEA15
:10373000410C5FEA5C5CF6D14FF000000149704734
:103740000000FF070000F87F0EF1020E2EF0030EBE
:103750005EF8046B364205D4012A43EB030515F5E8
:10376000001F12D8012841EB010C1CF5001F0CD8DA
:103770000ED14FEAD17C15F5001F0CEB4C0C0CF16F
:10378000020C08BF4CEBD37C04E04FF0080C01E0C6
:103790004FEAD37C0CEB4C0526FA05F606F007063B
:1037A000B6F1040C06D20EEB860CBDE870404CF06E
:1037B000010C6047DFE80CF0090B02024FF00041FA
:1037C0004FF00000A1F5002170BD194610460128F8
:1037D00051EB010418BFD4F5001484BF002001F0A0
:1037E000004170BD0808A0F500114FEA3101704793
:1037F00043004FEAD30C4FEA3C0C43401FBF400745
:103800000CF1605113F0FE4F70471CF0006F03D1B4
:1038100000200CF0004170470CF0004343EA507068
:1038200010B540EACC0000F027F800BF000000927D
:103830004FEA0001FFF7D6BF4FF000414FF0000004
:10384000A1F500217047000010F0004148BF404240
:10385000B0FA80F310FA03F2C3F19D030BD051EAE2
:10386000C35101EB1220530638BF704700F101002D
:1038700008BF20F0010070470EF1020E2EF0030E7B
:103880005EF8044B244204D44FEA4102B2F17F4F68
:1038900011D84FEA4003B3F17F4F0CD80ED14FEA55
:1038A000D07CB2F17F4F0CEB4C0C0CF1020C08BF3A
:1038B0004CEBD17C04E04FF0080C01E04FEAD17CE6
:1038C0000CEB4C0324FA03F404F00704B4F1040CE9
:1038D00006D20EEB840CBDE810404CF0010C6047A2
:1038E000DFE80CF0070802024FF00040A0F580006E
:1038F00010BD0846420018BFD2F1807288BF00F0A8
:10390000004010BD0000000000000000002F00007B
:1039100000000700070000147F147F1400242A7F92
:103920002A12006264081323003649552250000011
:103930000503000000001C224100000041221C0081
:103940000014083E08140008083E0808000000A003
:1039500060000008080808080000606000000020FF
:1039600010080402003E5149453E0000427F4000DD
:10397000004261514946002141454B310018141263
:103980007F10002745454539003C4A494930000130
:103990007109050300364949493600064949291E7F
:1039A00000003636000000005636000000081422E1
:1039B00041000014141414140000412214080002E1
:1039C0000151090600324959513E007C1211127C06
:1039D000007F49494936003E41414122007F414133
:1039E000221C007F49494941007F09090901003E25
:1039F0004149497A007F0808087F0000417F410063
:103A0000002040413F01007F08142241007F4040D8
:103A10004040007F020C027F007F0408107F003EC0
:103A20004141413E007F09090906003E4151215EA6
:103A3000007F091929460046494949310001017FA3
:103A40000101003F4040403F001F2040201F003F39
:103A50004038403F006314081463000708700807EB
:103A600000615149454300007F41410000552A55FE
:103A70002A55000041417F00000402010204004079
:103A8000404040400000010204000020545454789B
:103A9000007F4844443800384444442000384444BB
:103AA000487F00385454541800087E090102001859
:103AB000A4A4A47C007F080404780000447D400096
:103AC000004080847D00007F102844000000417F7A
:103AD0004000007C04180478007C08040478003856
:103AE0004444443800FC242424180018242418FCDE
:103AF000007C0804040800485454542000043F4447
:103B00004020003C4040207C001C2040201C003C09
:103B10004030403C004428102844001CA0A0A07C59
:103B2000004464544C441414141414140000000091
:103B3000000000000000000000000000000000F88D
:103B400000000000000000333000000000100C06F0
:103B5000100C0600000000000000000040C078408B
:103B6000C0784000043F04043F040400007088FC57
:103B700008300000001820FF211E0000F008F000AF
:103B8000E018000000211C031E211E0000F0088820
:103B9000700000001E2123241927211010160E008A
:103BA000000000000000000000000000000000E035
:103BB000180402000000000718204000000204184A
:103BC000E00000000040201807000000404080F0A6
:103BD000804040000202010F01020200000000F0DC
:103BE000000000000101011F0101010000000000B0
:103BF0000000000080B07000000000000000000025
:103C000000000000000101010101010100000000AD
:103C10000000000000303000000000000000000044
:103C200080601804006018060100000000E0100821
:103C30000810E000000F102020100F00001010F8F6
:103C4000000000000020203F202000000070080835
:103C500008887000003028242221300000300888B5
:103C6000884830000018202020110E000000C020DD
:103C700010F8000000070424243F240000F80888FE
:103C8000880808000019212020110E0000E010888B
:103C900088180000000F112020110E0000380808BD
:103CA000C83808000000003F0000000000708808CD
:103CB00008887000001C222121221C0000E010084E
:103CC0000810E0000000312222110F00000000C0A7
:103CD000C000000000000030300000000000008044
:103CE0000000000000008060000000000000804034
:103CF000201008000001020408102000404040404D
:103D0000404040000404040404040400000810209F
:103D100040800000002010080402010000704808E4
:103D20000808F0000000003036010000C030C8284C
:103D3000E810E0000718272423140B000000C03807
:103D4000E0000000203C23020227382008F8888881
:103D500088700000203F202020110E00C03008088D
:103D600008083800071820202010080008F8080864
:103D70000810E000203F202020100F0008F888885D
:103D8000E8081000203F20202320180008F8888829
:103D9000E8081000203F200003000000C0300808A1
:103DA0000838000007182020221E020008F808002A
:103DB0000008F808203F210101213F20000808F8F1
:103DC000080800000020203F202000000000080814
:103DD000F8080800C08080807F00000008F888C0D4
:103DE00028180800203F20012638200008F8080085
:103DF00000000000203F20202020300008F8F800BC
:103E0000F8F80800203F003F003F200008F830C0CD
:103E10000008F808203F200007183F00E0100808BD
:103E20000810E0000F10202020100F0008F80808EC
:103E30000808F000203F210101010000E0100808FF
:103E40000810E0000F18242438504F0008F8888824
:103E500088887000203F2000030C30200070880804
:103E6000080838000038202121221C00180808F812
:103E7000080818000000203F2000000008F8080093
:103E80000008F808001F202020201F000878880064
:103E900000C83808000007380E010000F80800F8D4
:103EA0000008F800033C0700073C0300081868807E
:103EB0008068180820302C03032C30200838C800F4
:103EC000C83808000000203F200000001008080843
:103ED000C83808002038262120201800000000FEE5
:103EE000020202000000007F40404000000C30C091
:103EF00000000000000000010638C00000020202BD
:103F0000FE000000004040407F000000000004026E
:103F10000202040000000000000000000000000099
:103F20000000000080808080808080800002020489
:103F30000000000000000000000000000000808081
:103F4000808000000019242222223F2008F80080EF
:103F500080000000003F112020110E0000000080B2
:103F600080800000000E1120202011000000008041
:103F70008088F800000E112020103F200000808073
:103F800080800000001F222222221300008080F087
:103F9000888888180020203F2020000000008080B2
:103FA00080808000006B94949493600008F80080F7
:103FB00080800000203F210000203F200080989852
:103FC000000000000020203F2020000000000080B2
:103FD0009898000000C08080807F000008F80000F2
:103FE00080808000203F24022D302000000808F847
:103FF000000000000020203F202000008080808002
:1040000080808000203F20003F20003F8080008093
:1040100080800000203F210000203F2000008080A1
:1040200080800000001F202020201F008080008052
:104030008000000080FFA12020110E000000008001
:1040400080808000000E112020A0FF8080808000F2
:104050008080800020203F2120000100000080801F
:10406000808080000033242424241900008080E014
:10407000808000000000001F2020000080800000E1
:1040800000808000001F202020103F2080808000C2
:104090000080808000010E300806010080800080D2
:1040A000008080800F300C030C300F0000808000F7
:1040B000808080000020312E0E3120008080800022
:1040C0000080808080818E701806010000808080D2
:1040D000808080000021302C222130000000000070
:1040E000807C020200000000003F40400000000011
:1040F000FF00000000000000FF0000000002027C42
:10410000800000000040403F000000000006010168
:104110000202040400000000000000003C4100080E
:1041200000000020840400006C01000848430008DF
:1041300084040020A4060000D0010008E200016011
:1041400004A24A040B100D0102030406070809002B
:1041500000C0381AF007FF000040201831F01200AC
:104160000080814020100C0300030C102040808050
:1041700020100A100C04C4040405F6040100041005
:10418000C4140C402004804241410005130C10224D
:104190004140000E101010FF109000FE82828292AB
:1041A000A29E8010060444827F01A0000710804375
:1041B0002C102C4340F01012EAAFAAEA0FFA028842
:1041C0008C5724548C844010070202EAAAAAAB023E
:1041D0001101000411EA0202A0000D109E929292B9
:1041E0009EE0809EB2D2929EE00010100808F494E7
:1041F0009292F10001F2929494F808C010076002C4
:104200008C0000FE440404119292FE40100A040443
:104210007E01407E42427E02040411427E406220C2
:1042200009FC242424FC25262408F60440040E114D
:1042300040308F80844C55252525554C8040100CEE
:10424000807000FF1008FE424242FA04011082040E
:104250001011806018070810FF50484641424C403A
:10426000FFC01007055555D5057F0607115505C038
:1042700015A0100A8AA96B352525ABE9080C051392
:1042800000040B14201808C838CF08082898000428
:104290000B50040201FF4021060A11200035804521
:1042A0007F051780000B124448507F40407F5048E4
:1042B00044802A7EFE00071040300F0414647F47BC
:1042C0000040BD31040004157E4040800009140206
:1042D000F202FE00F800FF80000B108047300F1044
:1042E000270047807F602009060909E6F80C0402D0
:1042F000010B11041E4120080000071F302040015F
:10430000031220101F13FE2201410501143F215BFF
:1043100022FF050E1207E00329401405180C24247F
:10432000820E1224C0032940000C1E9041310F015F
:10433000013F41417100012D58046D5C04000500EE
:08434000020406080000000061
:0400000508000131BD
:00000001FF
